:100000000C94D8020C9410030C9410030C9410035D
:100010000C9410030C9410030C9410030C94100314
:100020000C9410030C9410030C9429280C94FB28B6
:100030000C9408230C9410030C9410030C941003DC
:100040000C9410030C9410030C9410030C941003E4
:100050000C9410030C9490230C9410030C94100334
:100060000C9410030C9410030C9410030C941003C4
:100070000C9410030C9410030C9410030C941003B4
:100080000C9410030C9410030C9410030C941003A4
:100090000C9410030C9410030C9410030C94100394
:1000A0000C9410030C9410030C941003E805E8055D
:1000B000140614067C069A06B207B207A5063E0788
:1000C0004F074F0768298F29872A8F29872ADB291D
:1000D000FE29872A552A642A29001E001F002000B5
:1000E00021002200230024002500260027002D00E7
:1000F0002E0031002B0014001A0008001500170014
:100100001C0018000C00120013002F0030003500F6
:10011000390004001600070009000A000B000D005A
:100120000E000F003300340028002A00E1001D00FB
:100130001B000600190005001100100036003700F2
:100140003800E10035410000E000E300E20000007B
:10015000000000000000000000000000000000009F
:1001600000000000000000000000000000002C0063
:100170000000000000000000E600E700E4000000CE
:10018000005C3A003B003C003D003E003F00400068
:10019000410042004300440045000100010001000D
:1001A0000100010001000100010001000100010047
:1001B0000100520001000100010001000100C35CC8
:1001C000C45CC65CC75CC85CC95CCA5C50004F00BC
:1001D00001004C00010001000100C05CBE5CBF5C7E
:1001E000C15C01000100010051000100010000009C
:1001F00001000100010000000000000000000000FC
:1002000000000000000000000000000000000000EE
:1002100000000000000001000000000000000000DD
:10022000010001000100000000047F3F1F64321440
:10023000643214783C1E1E140A0522232526282920
:100240002A2C2D2F3032333536383A3B3D3E404252
:10025000434547494A4C4E5051535557595A5C5E95
:100260006062646668696B6D6F71737577797B7DA9
:100270007F81838587898A8C8E90929496989A9CA8
:100280009E9FA1A3A5A7A8AAACAEAFB1B3B4B6B8C0
:10029000B9BBBCBEBFC1C2C3C5C6C7C9CACBCCCD22
:1002A000CED0D1D2D2D3D4D5D6D7D7D8D9D9DADAFD
:1002B000DBDBDBDCDCDCDCDCDDDDDDDDDCDCDCDC7D
:1002C000DCDBDBDBDADAD9D9D8D7D7D6D5D4D3D2B1
:1002D000D2D1D0CECDCCCBCAC9C7C6C5C3C2C1BF8F
:1002E000BEBCBBB9B8B6B4B3B1AFAEACAAA8A7A5F3
:1002F000A3A19F9E9C9A98969492908E8C8A8987AF
:100300008583817F7D7B79777573716F6D6B69688C
:10031000666462605E5C5A5957555351504E4C4A60
:100320004947454342403E3D3B3A3836353332300B
:100330002F2D2C2A292826252322FFAA7F5540006D
:100340000101010101010101010202020202020296
:100350000202030303030303030304040404040469
:10036000040505050505060606060607070707072F
:1003700008080808090909090A0A0A0B0B0B0C0CE2
:100380000C0D0D0D0E0E0E0F0F0F1010111111127E
:100390001213131414151516161717181819191AFD
:1003A0001A1B1B1C1D1D1E1E1F2020212222232460
:1003B00024252626272829292A2B2C2D2D2E2F309F
:1003C000313232333435363738393A3B3C3D3E3FB3
:1003D000404142434445464748494A4C4D4E4F50A0
:1003E000515354555658595A5B5D5E5F616264655E
:1003F0006668696B6C6D6F7072737577787A7B7DE8
:100400007E8082838587888A8C8E8F91939596983B
:100410009A9C9EA0A2A3A5A7A9ABADAFB1B3B5B757
:10042000BABCBEC0C2C4C6C9CBCDCFD1D4D6D8DB2E
:10043000DDDFE2E4E7E9EBEEF0F3F5F8FAFDFF0CBF
:10044000035400520036003000570000001A0354D5
:10045000007200690061006E0067006C0065005F5B
:10046000004C006100620000000403090409023B23
:1004700000020100A0FA09040000010301010009C3
:100480002111010001224000070581030800010934
:10049000040100010300000009211101000122B63E
:1004A000000705820320000112010002000000087D
:1004B000EDFE404101000102000105010902A10118
:1004C00085020901A1000509190129081500250166
:1004D0009508750181020501093009311581257FD3
:1004E00095027508810609381581257F95017508E3
:1004F0008106050C0A38021581257F950175088152
:1005000006C0C005010980A101850319012AB700B1
:10051000150126B700950175108100C0050C090171
:10052000A101850419012AA002150126A002950146
:1005300075108100C005010906A10185060507198E
:10054000E029E715002501950875018102050719C5
:100550000029EF1500250195F075018102050819A4
:10056000012905950575019102950175039101C059
:1005700005010906A101050719E029E71500250174
:10058000950875018102950175088101050719001B
:1005900029FF150026FF009506750881000508193A
:1005A000012905950575019102950175039101C019
:1005B00011241FBECFEFDAE0DEBFCDBF04B603FECD
:1005C00018C08091260390912703A0912803B09131
:1005D00029038730904BA740B04B59F41092260363
:1005E000109227031092280310922903E0E0F8E309
:1005F000099511E0A0E0B1E0E0E6F7E502C0059062
:100600000D92A83CB107D9F723E0A8ECB1E001C0F6
:100610001D92A632B207E1F70E94C4130C94AE2BD0
:100620000C940000CF93C82F0E94FF03882379F019
:10063000C0FD02C0299A01C02998C1FD02C02A9AB2
:1006400001C02A98C2FD02C02B9A01C02B98CF91FD
:10065000089581E0089581E008950C942B03089596
:100660000C942F031F93CF93DF9300D000D01F92E1
:10067000CDB7DEB749835A836B833091CB01898133
:100680009A81311114C0662359F0222349F00E9447
:10069000EF09182F682F89819A810E94980903C059
:1006A0000E94C309182F69817A81812F04C00E949A
:1006B000EF0969817A810F900F900F900F900F9042
:1006C000DF91CF911F910C942F11FC01262F4081B7
:1006D00051816281738184810C94320381E0089599
:1006E000CF93DF93EC0160E00E946503BE01DF91D0
:1006F000CF910C9430030C9475120C9471120895E0
:100700000E9442080E947F032FEF84E39CE0215067
:1007100080409040E1F700C000000C94B6230F9396
:100720001F93CF93DF938C0161E00E946503EC017E
:10073000B8010E942D03882309F44BC0B801CE01F3
:100740000E94411E882309F444C0B801CE010E94D2
:1007500053218823F1F1B801CE010E94671F88233D
:10076000C1F1B801CE010E94AF20882391F1B801F8
:10077000CE010E94851C882361F1F80182818823C3
:1007800009F1CB358DE5D807C1F050F4C115FCE572
:10079000DF0781F0CF3DDC45A9F40E94260F19C088
:1007A000CC35EDE5DE0761F0CD35DD4559F40E942D
:1007B000690E08C00E9480030CC00E94720E02C025
:1007C0000E94750EC801DF91CF911F910F910C947B
:1007D000290380E0DF91CF911F910F9108950E942E
:1007E000EA2280E00E94761E0C940B040E94651D94
:1007F0000E940E040C94F02208950C94FC0381E0F6
:1008000008950895CF93C82F0E94FD038C2F0E9456
:100810001203CF91089580E00C9402040E94AF214E
:100820000C9402040E94AF219091CA01891721F013
:100830008093CA010C9402040895CF93DF93CDB73F
:10084000DEB72B970FB6F894DEBF0FBECDBF4F8338
:10085000588769877A878B8761110E94B50D9E0141
:100860002F5F3F4F86E0F90111928A95E9F785E005
:10087000FE013796D90101900D928A95E1F78981A1
:100880009A814C815D81452B31F09F3F31F491E09D
:100890008F3F19F403C091E001C090E090FF09C0C0
:1008A00049815A816B817C818D819E810E94D60C09
:1008B00005C0C9010E946E038111F2CF2B960FB6BD
:1008C000F894DEBF0FBECDBFDF91CF910895FC013C
:1008D000808191810E94310A0895CF93882309F481
:1008E000A4C0C82F8238C1F40E94AF2181FD9DC0F1
:1008F00069E380910201909103010E94A5220E9468
:10090000D70D2FEF81EE94E0215080409040E1F729
:1009100000C0000069E319C0833801F50E94AF21CF
:1009200080FD83C063E580910201909103010E94E4
:10093000A5220E94D70D2FEF81EE94E02150804038
:100940009040E1F700C0000063E5809102019091C2
:1009500003010E94B022CF910C94D70D8438C1F4CA
:100960000E94AF2182FD61C067E4809102019091F5
:1009700003010E94A5220E94D70D2FEF81EE94E083
:10098000215080409040E1F700C0000067E4DDCFD7
:100990008CEF8C0F813AD0F46C2F809102019091F2
:1009A00003010E942522882349F06C2F80910201C7
:1009B000909103010E94B0220E94D70D6C2F80916C
:1009C0000201909103010E94A522C5CF80E28C0F05
:1009D000883048F4C77081E001C0880FCA95EAF7F3
:1009E0000E94980DB8CFEBE5EC0FE33040F4F0E057
:1009F000E65AFE4F808190E0CF910C94E321E8E528
:100A0000EC0FE73150F4F0E0EE0FFF1FE45DFE4F16
:100A100080819181CF910C94F921CD3E30F08C2FC3
:100A20000E944914CF910C941B15CF9108958823EF
:100A300009F464C0823879F40E94AF2181FF5EC05E
:100A400069E380910201909103010E94A5220E9416
:100A5000D70D69E310C08338B1F40E94AF2180FF45
:100A60004DC063E580910201909103010E94A5228F
:100A70000E94D70D63E580910201909103010E94CD
:100A8000B0220C94D70D843879F40E94AF2182FFF4
:100A900035C067E480910201909103010E94A52274
:100AA0000E94D70D67E4E7CF9CEF980F913A10F4BE
:100AB000682FE1CF90E2980F983050F4877091E062
:100AC00001C0990F8A95EAF7892F0E949E0DD9CF10
:100AD0009BE5980F933020F480E090E00C94E321A4
:100AE00098E5980F973120F480E090E00C94F9217C
:100AF0008D3E20F00E94A4140C941B1508951F93A2
:100B0000CF93DF93182FEB010E946D04209741F0E3
:100B10008FE99FE00197F1F700C000002197F6CF21
:100B2000812FDF91CF911F910C941705893319F014
:100B300060E070E002C060E570E00C947F058823FF
:100B400021F00E94980D0C94D70D0895882321F070
:100B50000E949E0D0C94D70D0895CF92DF92EF92D4
:100B6000FF920F931F93CF93DF937C01D62FC72F54
:100B7000FC011281058102950F700E948E0D882361
:100B8000B9F01123A9F08C2F807F803421F080E20E
:100B90008D0F883068F08091EA0282FD09C082E002
:100BA0000E94370E0E948E0D91E0D82ED92601C0EA
:100BB000D12CCC2EC2948FE0C8228C2D90E08C30AA
:100BC000910508F0CFC1FC01EA5AFF4F0C94152B98
:100BD0008C2F807FCF70882311F0C295C07F1123A6
:100BE00099F0CC2309F4AAC180E28D0F883010F06F
:100BF000D11104C08C2F0E94980D03C08C2F0E942D
:100C0000A80D0E94D70D9AC18D2F0E941705CC23E5
:100C100009F4A8C180E28D0F883038F1DD2329F175
:100C20008C2F0E94AE0D24C08C2F807FCF7080321D
:100C300011F0C295C07FDD2319F0D130A1F13DC084
:100C40008091EA0282FF17C0112349F0CC2329F0DA
:100C50008C2F0E94980D0E94D70D80E070C180E01B
:100C60000E941705CC2309F47DC18C2F0E949E0D94
:100C70000E94D70D77C1112371F0002341F001309C
:100C800031F40E94B80D8C2B0E94C00D6BC10E94E4
:100C9000B80D8C2B1DC0002319F0013009F462C17E
:100CA0000E94CD0D25C0112321F0063008F05AC155
:100CB0000EC0053008F056C11BC0112361F000239F
:100CC00031F0F701858180FF39C18F7085838C2FCA
:100CD0000E949F0547C1002359F0D93309F03FC155
:100CE000FFEF07EE13E0F15000401040E1F735C18F
:100CF0008C2F0E94A60536C18C2F86958695837011
:100D000019F0813061F02EC1112321F08D2F9C2F1D
:100D1000937002C080E090E00E94E3212BC1112378
:100D200021F08D2F9C2F937002C080E090E00E94F4
:100D3000F92120C18D2F112319F00E94491402C0FE
:100D40000E94A4140E941B1515C18C2F837009F0FA
:100D500047C011110BC12D2F229526952770220F08
:100D6000220F6D2F6F70862F90E0A0E0B0E0022E72
:100D700004C0880F991FAA1FBB1F0A94D2F7D4FF83
:100D800010C04FE050E060E070E004C0440F551F19
:100D9000661F771F2A95D2F74095509560957095FC
:100DA00003C040E050E0BA01C695C695C3708A0101
:100DB0009B01082B192B2A2B3B2BC901B801C230F0
:100DC00049F058F4C13019F00E94AE08CFC00E941B
:100DD0009C08CCC00E94C008C9C00E949A08C6C026
:100DE000112319F08C2F817001C08695882309F496
:100DF000BDC02D2F229526952770220F220F6D2F13
:100E00006F70862F90E0A0E0B0E0022E04C0880F43
:100E1000991FAA1FBB1F0A94D2F7D4FF10C04FE03E
:100E200050E060E070E004C0440F551F661F771F5C
:100E30002A95D2F7409550956095709503C040E093
:100E400050E0BA01C695C695C3708A019B01082B74
:100E5000192B2A2B3B2BC901B801C23049F058F499
:100E6000C13019F00E94730981C00E9461097EC0DF
:100E70000E9485097BC00E94D40878C0CF701123DE
:100E800039F08C2F0E94FA088D2F0E949F056EC0AA
:100E90008D2F0E94A6058C2F0E941B0967C0D23F90
:100EA00021F128F4D03F41F0D13FC1F043C0D33FFE
:100EB00019F1D43F79F03EC0112341F0053008F01C
:100EC00051C08C2F8F710E9440094CC0063008F031
:100ED00049C0F7CF8091EA0282FF18C0112339F090
:100EE0008C2F8F710E94FA083DC01123C9F38C2FFB
:100EF0008F710E941B0936C0112329F08C2F8F712E
:100F00000E94E5082FC00E94E0082CC0112349F080
:100F1000CF718C2F0E94FA0863E08C2F0E941C0E68
:100F200021C081E00E94370E0230E0F082E00E9492
:100F3000370E18C0112331F0002391F28D2F0E943B
:100F40006D0410C0002399F2D93349F41FEF27EE46
:100F500033E0115020403040E1F700C000008D2FF9
:100F60000E94170588EF8C0D843020F40E94AF2179
:100F70000E940204DD20C9F00E948A0D80FD15C088
:100F8000F70112820E94840D0E94FA08C7010E9494
:100F9000F6070E94840DDF91CF911F910F91FF9072
:100FA000EF90DF90CF900C941B09DF91CF911F91B0
:100FB0000F91FF90EF90DF90CF9008950F931F93C4
:100FC000CF93DF93EC01688179818A810E943C0A8A
:100FD0008C010E9497090E948808B801CE010E94E6
:100FE000AD05DF91CF911F910F910895CF93DF93BE
:100FF000EC01988189812B813C81232B31F08F3F3B
:1010000031F481E09F3F19F403C081E001C080E02A
:1010100080FD1DC0CE010E948F03811110C00E946F
:101020008E0D8823A1F08A81882389F08091EA02BD
:1010300082FD0DC082E0DF91CF910C94370ECE017E
:101040000E94DE07CE01DF91CF910C947003DF91F7
:10105000CF91089580E090E00E94E32180E090E04D
:101060000E94F9210E94B50D0E94D70D0E944C16D6
:101070000C941B1580910201909103010E94BB22E8
:101080000C942A080E94A50D0C943A0892959F7022
:10109000963079F010F4925001C09A50923068F472
:1010A000803F69F018F4883E40F409C0843F29F479
:1010B00006C0883E20F0813F11F080E0089581E075
:1010C0000895FC01808191810E94310A0E944608A6
:1010D0000895CF93DF9300D000D01F92CDB7DEB735
:1010E0000F900F900F900F900F90DF91CF91089578
:1010F000CF93DF9300D000D000D0CDB7DEB72696D7
:101100000FB6F894DEBF0FBECDBFDF91CF9108952B
:10111000089508950C9489080C948A080E948C08FC
:1011200060930702709308028093090290930A0269
:101130000C942A080C948E080F931F9300910702B9
:10114000109108022091090230910A02602B712B44
:10115000822B932B1F910F910C948E080F931F934A
:1011600000910702109108022091090230910A02B1
:1011700060237123822393231F910F910C948E0877
:101180000F931F930091070210910802209109020A
:1011900030910A0260277127822793271F910F91B0
:1011A0000C948E080C9489080E94D2086093030264
:1011B0007093040280930502909306020C942A080F
:1011C00060E070E0CB010C94D4080F931F9341E0D2
:1011D00050E060E070E08A019B0104C0000F111F25
:1011E000221F331F8A95D2F7C901B8011F910F91B1
:1011F0000C94D4080F931F9341E050E060E070E03E
:1012000004C0440F551F661F771F8A95D2F780913F
:10121000030290910402A0910502B09106028A0196
:101220009B01082B192B2A2B3B2BC901B8011F91BD
:101230000F910C94D4080F931F9341E050E060E0AD
:1012400070E004C0440F551F661F771F8A95D2F7C0
:10125000409550956095709580910302909104029D
:10126000A0910502B09106028A019B01082319236F
:101270002A233B23C901B8011F910F910C94D40874
:101280000F931F9341E050E060E070E004C0440F12
:10129000551F661F771F8A95D2F7809103029091A0
:1012A0000402A0910502B09106028A019B01082761
:1012B00019272A273B27C901B8011F910F910C94C8
:1012C000D4080F931F930091030210910402209100
:1012D000050230910602602B712B822B932B1F91FC
:1012E0000F910C94D4080F931F9300910302109157
:1012F00004022091050230910602602371238223AB
:1013000093231F910F910C94D4080F931F93009176
:101310000302109104022091050230910602602719
:101320007127822793271F910F910C94D408089559
:101330002EE0929F800D1124E82FE695E695E69524
:10134000877051E001C0550F8A95EAF785E0E89F64
:10135000F0011124E453FE4F20E030E070E04081C2
:10136000CB01022E02C0969587950A94E2F7817010
:10137000819584278523842781932F5F3F4F2530D4
:10138000310569F708952EE0929F800D1124682F92
:10139000669566956695982F977085E0689FB00171
:1013A000112440E050E080E0FB01E40FF51FE4531E
:1013B000FE4F208130E0092E02C0369527950A9411
:1013C000E2F721703327042E01C0220F0A94EAF7B6
:1013D000822B4F5F5F4F4530510531F70895BF9223
:1013E000CF92DF92EF92FF920F931F93CF93DF93F1
:1013F0008C01C0900302D0900402E0900502F090AE
:1014000006028091070290910802A0910902B09112
:101410000A02C82AD92AEA2AFB2ACFE1D0E0D7015A
:10142000C6010C2E04C0B695A795979587950A948A
:10143000D2F780FD04C0219790F7B12C07C0BC2ED5
:10144000B8018C2F0E9442110197A9F38B2DDF91D7
:10145000CF911F910F91FF90EF90DF90CF90BF90B1
:101460000895CF93DF93EC010E94EF09BE010E9423
:101470004211DF91CF9108951F93CF93DF93EB013A
:101480009091CB01992321F0CB010E94310A13C026
:10149000882349F0CB010E94EF09182F682FCE0155
:1014A0000E94980904C0CB010E94C309182FBE01F5
:1014B000812F0E944211DF91CF911F9108951F93B8
:1014C000CF93DF93C0910B0216E080910C02C817F6
:1014D00099F0D0E01C9FF0011D9FF00D1124E35FF7
:1014E000FD4F4081518162817381848195810E9489
:1014F00078082196C770E9CFDF91CF911F910895A9
:1015000040913D0250913E0260913F027091400235
:1015100080914102909142020C947808EF92FF92E0
:101520000F931F93CF93DF938091420282958F7028
:1015300009F065C080913F02882309F460C0809162
:101540000B02F0900C0210913D0200913E0260915E
:1015500040027091410291E01F3F09F090E0C0917C
:101560000001D0910101292F96E0E92E8F1509F491
:1015700046C06115710521F00F3F21F030E003C036
:1015800031E001C0322F90E030FD36C0E89EF0011E
:10159000E99EF00D1124DF01A35FBD4F11963C9130
:1015A0001197301329C03C91311326C012963C91FB
:1015B0001297311121C013964D915C911497461BDF
:1015C000570B4C175D07C0F4809142028F70806109
:1015D00080934202EE5EFD4F80818F708061808338
:1015E0008DE392E00E94F607DF91CF911F910F915A
:1015F000FF90EF900C945F0A01968770B7CFDF9150
:10160000CF911F910F91FF90EF9008959F92AF920D
:10161000BF92CF92DF92EF92FF920F931F93CF93DF
:10162000DF93CDB7DEB761970FB6F894DEBF0FBE7C
:10163000CDBF8C0185E0F801DE011D9601900D9271
:101640008A95E1F7D8011296EC9090913D02E091D5
:101650003E0220914002309141022115310531F0C6
:10166000EF3F31F481E09F3F19F403C081E001C0F6
:1016700080E0B82FB1709B2E80FD47C1D8014C91FE
:1016800011965C9111971396AD90BC9014978DE3D1
:10169000C82E82E0D82EF0903F02B501621B730B7A
:1016A0002091000130910101FF2009F4D9C08091FF
:1016B00042026217730708F095C0282F207F09F0B7
:1016C00052C05E1313C0491311C0FE2CE1100EC0AE
:1016D0008F708061809342020E94800AC6010E943E
:1016E000F60780914202F80185834DC1AB2831F0A5
:1016F0005F3F31F481E04F3F19F403C081E001C046
:1017000080E080FD03C081E08E2502C080E090E093
:10171000F82FF170FF2E80FF1CC080910B022091EA
:101720000C0236E0821709F40BC190E0389FF001FB
:10173000399FF00D1124E35FFD4F6181561306C000
:101740006081461303C06281E61203C00196877070
:10175000E9CFFE2CEE2009F416C18091420281608F
:101760008093420254C05E1306C0491304C0E110C6
:1017700002C0F80199C0C8010E946108882361F184
:10178000EE2051F120914202822F82958F7090E0DD
:10179000029774F080913D0290913E0298878F836A
:1017A0001986BB86AA862C87CE0107960E94F6076B
:1017B00086E0F801ADE3B2E001900D928A95E1F781
:1017C0000E948E0A0E94800A0AC05E1711F1C801A9
:1017D0000E94610881112CC0C8010E94F607FF24F5
:1017E000F394D1C0282F207F81F77A2DB98AA88A57
:1017F0006E2D89890E9469088DE392E00E94F607A8
:1018000086E0D6011D928A95E9F70E94800AF12CA4
:10181000BAC04913DCCFE110DACFF8018583C801E3
:101820000E94F60786E0D6011D928A95E9F7ABC0C3
:10183000EE2091F220914202822F82958F7090E0EB
:1018400002970CF4B5CF80913D0290913E029A83AD
:1018500089831B82BD82AC822E83CE010196A6CFE6
:101860006217730708F044C0FE2CEE2009F4B4CFD1
:101870005E1330C049132EC02091420220FD21C0CA
:10188000822F82958F70482F50E041155105C9F085
:10189000F80125834F30510541F08F5F982F9295C5
:1018A000907F822F8F70892B8583C8010E94F60755
:1018B00086E0F801ADE3B2E001900D928A95E1F780
:1018C0003CC086E0F801ADE3B2E001900D928A954C
:1018D000E1F759C0C8010E946108811169CF809168
:1018E0004202816080934202C8010E94F6074BC009
:1018F0007A2DB98AA88A6E2D89890E94690886E0A6
:10190000D6011D928A95E9F718C0EE2009F464CF3C
:10191000C8010E946108F82E882309F45DCF86E093
:10192000F801ADE3B2E001900D928A95E1F78DE305
:1019300092E00E9467040E948E0A0E94800A23C0DF
:101940004D875E878D859E850E94310A292F2295BD
:101950002F70223028F49F7039F0811105C00BC020
:10196000243028F49F7049F4805E883020F0C8014C
:101970000E94F6079F2CF92C06C0D80115969C9161
:10198000907F91F7F8CF8F2D61960FB6F894DEBF58
:101990000FBECDBFDF91CF911F910F91FF90EF90C0
:1019A000DF90CF90BF90AF909F9008951F93CF93FB
:1019B000DF93CDB7DEB72C970FB6F894DEBF0FBE1E
:1019C000CDBF4F83588769877A878B879C87CE01E5
:1019D00007960E94060B8823D1F09F8188852A856F
:1019E0003B85232B31F08F3F31F481E09F3F19F489
:1019F00003C081E001C080E080FD47C04F81588571
:101A000069857A858B859C850E9478083EC086E032
:101A1000FE013796DE01119601900D928A95E1F74D
:101A2000FF81E8856A857B856115710531F0EF3F9F
:101A300031F481E0FF3F19F403C081E001C080E090
:101A400080FD23C020910C0230E0C901019687700F
:101A5000992740910B0250E084179507F1F1F98323
:101A6000EA837D836C8396E0929FD001939FB00DB3
:101A70001124A35FBD4FFE01319601900D929A95FE
:101A8000E1F780930C020E945F0A16E080910B023E
:101A900090910C02891771F1189FC0011124835F86
:101AA0009D4F0E94060B882329F1E0910B021E9F97
:101AB000F0011124E35FFD4F408151816281738108
:101AC000848195810E94780880910B0290E00196B4
:101AD0008770992780930B02D9CF0E9442081092F9
:101AE0000C0210920B02EDE3F2E086E0DF011D92A2
:101AF0008A95E9F72C960FB6F894DEBF0FBECDBFDE
:101B0000DF91CF911F91089580916302859585950E
:101B1000859508958091630287700895909163027E
:101B2000977081E009F480E008958091860208951D
:101B300090918602892B80938602089580959091DA
:101B40008602892380938602089510928602089562
:101B500090918502892B80938502089580959091BC
:101B60008502892380938502089510928502089545
:101B700080916402089508950C94BB0D0C94BC0DE3
:101B80009091EA0292FD08C090916402981721F0AA
:101B9000809364020C94BE0D0895809164028823A2
:101BA00029F01092640280E00C94BE0D0895CF934A
:101BB000DF93E0910201F09103018091860280831E
:101BC000E0910201F0910301908180918502892BBF
:101BD000808380916402882381F0E0910201F0917A
:101BE00003019081892B80838091020190910301F0
:101BF0000E940F2281110E94CD0DC0910201D0914F
:101C0000030140E250E063E472E0CE010E94592BF0
:101C1000892B69F080E2FE01A3E4B2E001900D920D
:101C20008A95E1F7CE01DF91CF910C94BB21DF9132
:101C3000CF9108950C94BB0D9091EA0292FD10C0D3
:101C400098E0899F90011124262B209363020E9423
:101C5000FA08809163028595859585950C941A0EF6
:101C60000C94FA081092630280E00C941A0E2091F2
:101C700063028095822380936302982F977099F472
:101C800030E0482F082E000C550B2417350759F06B
:101C90009091EA0292FD07C08595859585950E94F1
:101CA0001B090C94320E08959091EA0292FB2227B0
:101CB00020F9281769F080FB92F99093EA0280914D
:101CC000E9029091EA020E94A20E82E00C94370E83
:101CD00008958091EA0282FB882780F991E08927A4
:101CE0000C94540E81E00C94540E80E00C94540E2D
:101CF0006FEF7FEF80E090E00C94982B80E090E015
:101D00000E94742B21E0893E9E4F09F020E0822F33
:101D1000089582E090E00C94662B83E090E00C94B0
:101D2000662BCF9384E090E00E94662BC82F82E25E
:101D300090E00E94662B2C2F30E0A901582BCA019D
:101D4000CF910895CF93C92F682F84E090E00E942F
:101D50007A2B6C2F82E290E0CF910C947A2BAB011E
:101D6000BC018FE090E00C948C2BAB01BC0183E1B3
:101D700090E00C948C2B60E070E0CB010C94B50EDD
:101D800060E070E0CB010E94AF0E0C94BB0E69EED8
:101D90007EEF80E090E00E94982B60E082E090E08F
:101DA0000E947A2B60E083E090E00E947A2B1092F0
:101DB0000702109208021092090210920A0260E0D3
:101DC00084E090E00E947A2B60E082E290E00E9442
:101DD0007A2B60E085E090E00E947A2B60E086E05C
:101DE00090E00E947A2B6FEF87E090E00E947A2BC0
:101DF00040E050E0BA0188E090E00E948C2B60E067
:101E00008DE090E00E947A2B40E050E0BA0188E13A
:101E100090E00E948C2B60E087E190E00E947A2B9A
:101E200040E050E0BA018CE190E00E948C2B60E031
:101E300070E080E290E00E94982B40E050E0BA0110
:101E400088E190E00E948C2B0C94C00E0C94C70E7D
:101E5000682F8EE090E00C947A2B0E94752360939B
:101E60009702709398028093990290939A026093DC
:101E70009302709394028093950290939602089532
:101E800085B7806885BF85B7806885BF089581E084
:101E900008950C94470F08950C944B0F0C944B0F1E
:101EA0000C944E0F0C944B0F0C94520F0C944B0F40
:101EB0000E94400F8EE192E10E94A5210E94560FE0
:101EC0000C94540F0E944C0F0C944B0F0E9438122C
:101ED0000E9401040C942C1F0E9460230E941D1379
:101EE0000E94660F0E94651D0E94A41B0C94500F57
:101EF0005F926F927F928F929F92AF92BF92CF929A
:101F0000DF92EF92FF920F931F93CF93DF93CDB7A2
:101F1000DEB72A970FB6F894DEBF0FBECDBF0E9482
:101F20003213C82E81110E942D0F37E8832E32E024
:101F3000932E00E010E0502E802F0E945C125C0176
:101F4000F401619071904F01682679266114710443
:101F5000B1F40F5F1F4F0630110569F78FEF8983CA
:101F60008A831B820E9469238160782F9D838C83E2
:101F700049815A816B818D810E941D043AC08091F4
:101F80009B0281FD0E946512D12CEE24E394F12C7A
:101F9000C3018E219F21892B29F10E94490F88239B
:101FA000A9F0DE825F82AE20BF2081E0AB2809F479
:101FB00080E088870E9469238160782F9A878987CB
:101FC0004E815F8168858A850E941D04000F111F64
:101FD000F801E957FD4F80819181E826F926F182C9
:101FE000E08207C0D394EE0CFF1CFEE0DF12D0CFDE
:101FF000B0CF81E0C11001C080E02A960FB6F894FE
:10200000DEBF0FBECDBFDF91CF911F910F91FF902B
:10201000EF90DF90CF90BF90AF909F908F907F9088
:102020006F905F9008950E94780F0E94D71B0E94C6
:102030002B1F0E9439150C941204CF93DF930E943A
:102040004711EC01811521E5920708F045C0811583
:1020500030E5930708F094C0883E910528F5803E4E
:10206000910508F0F8C0883A910570F4853A910519
:1020700008F07CC08130910509F475C008F4E8C00F
:10208000049708F0E8C0E4C08F3B910508F0E0C079
:10209000C85AD0E0CC0FDD1FC35ADE4F0990D8815B
:1020A000C02DCE019464D8C0811540E2940758F445
:1020B000811551E0950708F0CEC08D3E910508F4DA
:1020C000C7C09065C9C0C11580E4D80708F4C0C076
:1020D000DF70CE01906AC0C0811525E59207A8F493
:1020E000811534E5930708F095C0811543E5940701
:1020F00008F07BC0811552E5950708F061C0D82F24
:10210000CC27CE01816F906AA7C0C11589E5D80799
:10211000A0F4C11528E5D20708F082C0C11536E544
:10212000D30708F095C08C2F0E94DB118F7190E0CF
:10213000D82FCC27CE0190628FC0C1154AE5D407B5
:1021400008F474C0CE0190568115904208F080C00A
:102150008D2F8F710E94DB11DD27D0628F71AE0150
:10216000582BCA0179C081E090E076C0C55AD0E012
:10217000C557DE4F8881C82FD0E0CE0190646CC077
:1021800074E0969587957A95E1F7282F23703C2F78
:10219000337081E090E002C0880F991F3A95E2F712
:1021A0009C68AC01522B9A019C2F9F709695969536
:1021B00050E2959FE0011124C9018C2B9D2B4CC04E
:1021C0008370992721E030E002C0220F331F8A95E7
:1021D000E2F79C2F9695969580E2989FE001112456
:1021E000C22BD32BCE019C6837C08370992721E086
:1021F00030E002C0220F331F8A95E2F79C2F96959C
:10220000969540E2949FE0011124C22BD32BCE017E
:102210009A6822C0D82FCC27CE01846F906A1CC048
:10222000DC2FCC27CE01806F906A16C08C2F8F7068
:102230000E94DB1194E0D695C7959A95E1F7CF708F
:10224000D0E0DC2FCC27D0699E01282BC90104C027
:1022500080E090E001C0CE01DF91CF91089524E5A8
:10226000829FC0011124FC012EE0729FE00DF11D40
:102270001124E60FF11DEE0FFF1FE852FF4F85916D
:10228000949108950E942F110E941D100895823884
:10229000910569F1B0F48133910509F46DC048F4FA
:1022A0008932910509F463C08A32910509F469C045
:1022B00008958533910509F455C089339105B9F026
:1022C0000895833E910569F138F4803E9105B1F09F
:1022D000823E910509F10895863E9105A9F1873E58
:1022E0009105B9F1843E910509F064C023C02091A5
:1022F000E90220FD4FC021FD4DC008958091E90203
:1023000080FD44C08091EA0280FF44C08091E902D0
:1023100084FD42C083EE4DC08091E90282FF38C047
:10232000F5CF8091E90282FD33C08091EA0280FD01
:1023300031C0ECCF8091EA0281FF32C08091E90286
:1023400084FD2AC087EE35C08091E90283FF26C054
:10235000F5CF8091E90283FD21C08091EA0281FDE1
:102360001FC0ECCF8091E90285FD1CC01DC080918B
:10237000E90285FD19C016C08091E90286FD16C0EC
:1023800017C08091E90286FD13C010C089E311C017
:1023900082EE0FC080EE0DC080E00BC086EE09C05B
:1023A00084EE07C089E205C085E303C08AE201C06C
:1023B00081E390E008959091E90292FF0DC0282FEB
:1023C0002871283019F4877F846006C0282F247173
:1023D000243011F48B7F886093FF0DC0282F287163
:1023E000283119F4877E846106C0282F2471243196
:1023F00011F48B7E88612091EA0220FF0DC0382FF6
:102400003871383019F4877F816006C0382F3171F8
:10241000313011F48E7F886021FF0DC0282F287184
:10242000283119F4877E816106C0282F217121315E
:1024300011F48E7E886194FD877E089580E0089572
:102440000C94780E0E9432138FE39CE90197F1F708
:1024500000C000000E94321380E00E945C1280FFE6
:1024600004C00E9420120C94B62308950C942212EA
:102470000E947E0E811102C00E94260F0E94890ECA
:1024800080939B020E94910E9093EA028093E9024E
:102490000E9436120E948D0E682F70E080E090E05E
:1024A0000E949A08609103027091040280910502D3
:1024B000909106020C94D208E82FF0E0EE0FFF1F77
:1024C000E950FD4F808191810895089580EA8A95B1
:1024D000F1F7089500C008950C94661208950C94C5
:1024E0006E120C946F120C946E120C947312F8947A
:1024F000E82FE295EF70F0E031A1282F2F7081E0F6
:1025000090E001C0880F2A95EAF7982F90959323C1
:1025100091A392A1892B82A3789408950F931F937E
:10252000CF93DF93CCE9D1E089918F3F11F00E94E6
:10253000771281E0C23AD807B9F7CEE8D1E00CE9CA
:1025400011E089918F3F11F00E9477120C171D073F
:10255000C1F7DF91CF911F910F910895BF92CF9254
:10256000DF92EF92FF920F931F93CF93DF938C0133
:10257000C62FD0E0CE0184569E4F6C01FC019081A5
:102580009F3F09F450C0B62EF894E92FE295EF7002
:10259000F0E081A19F7021E030E001C0220F9A9508
:1025A000EAF7822B81A382A12095282322A3789485
:1025B0000E946A12EEE8F1E04CE951E021E030E0DF
:1025C000E12CF12C61916F3F89F0A62FA295AF709D
:1025D000B0E090968C9190E06F7002C095958795D1
:1025E0006A95E2F780FD02C0C90102C080E090E078
:1025F000E82AF92A220F331F4E175F0719F7F60151
:1026000080818F3F11F00E94771261E0E114F104A4
:1026100009F460E08B2D0E946C12CC0FDD1FC00FFF
:10262000D11FF982E882DF91CF911F910F91FF9026
:10263000EF90DF90CF90BF9008950E948E128CE0B3
:10264000E7EFF2E0DF01982F1D929A95E9F7EBEEA4
:10265000F2E0DF011D928A95E9F786E00E947D1382
:102660000C947B03FF920F931F93CF93DF93CDB70F
:10267000DEB72C970FB6F894DEBF0FBECDBF8E012C
:102680000F5F1F4F8CE0F80111928A95E9F7F12C4A
:102690006F2DC8010E94AE12F394F6E0FF12F8CF3E
:1026A0004CE050E0B8018BEE92E00E94592BFF24E1
:1026B000F394009709F4F12C892B41F08CE0F80198
:1026C000ABEEB2E001900D928A95E1F72F2D46E036
:1026D00067EF72E08BEE92E00E947E130E947D0312
:1026E0008F2D2C960FB6F894DEBF0FBECDBFDF91B5
:1026F000CF911F910F91FF9008950895FF920F932E
:102700001F93CF93DF93F82E092F162FD72FC42FA7
:10271000222349F081E080939E020E9469239093D6
:102720009D0280939C0280919E028823D9F0809123
:102730009C0290919D020E948123059798F0EF2DB5
:10274000F02FA12FBD2F80E090E04C2F50E0841798
:10275000950734F4219131912D933D930196F7CF54
:1027600010929E02DF91CF911F910F91FF900895DB
:102770000E9481250E946C0F0C948D250E9491254A
:102780000E9413100C94AB250E9407230E94682519
:102790000E94580F0E94B8130E94BE130E94620F3D
:1027A000FBCF8091A50280FF06C06091090170E017
:1027B000660F771F26C081FF04C06091090184E085
:1027C00005C082FF07C06091090188E0689FB001E1
:1027D000112417C09091A4029923D1F060910801AF
:1027E000961788F72091090188E0289F900111240D
:1027F000929FA001939F500D112470E0CA010E9486
:10280000DF2A6038710540F46115710519F406C0BE
:1028100068E070E0862F08958FE7089581E00895BD
:102820008091A50280FF08C06091050170E0759558
:1028300067957595679521C081FF06C06091050178
:1028400070E07595679519C082FF04C0609105011D
:1028500070E010C09091A302992399F06091040157
:102860009617A0F780910501899FC001112470E09F
:102870000E94DF2A6038710540F46115710519F472
:1028800006C061E070E0862F08958FE7089581E02B
:1028900008958D3E21F40E94D113819504C08E3E8F
:1028A00029F40E94D1138093A90208958F3E21F448
:1028B0000E94D113819504C0803F29F40E94D11356
:1028C0008093A8020895893F19F40E94101405C04E
:1028D0008A3F31F40E94101481958093AA020895D2
:1028E0008B3F21F40E941014819504C08C3F29F481
:1028F0000E9410148093AB0208959FE0980F9830C7
:1029000078F421E030E0A90102C0440F551F9A95E8
:10291000E2F7CA019091A702892B8093A70208953C
:102920008D3F21F48091A50281600BC08E3F21F480
:102930008091A502826005C08F3F29F48091A50295
:1029400084608093A50208958D3E39F49091A90288
:1029500097FF35C01092A90259C08E3E29F490917C
:10296000A9021916BCF32BC09091A8028F3E29F43E
:1029700097FF25C01092A80249C0803F19F419168C
:10298000CCF31DC09091AA02893F29F41916BCF41A
:102990001092AA023BC08A3F19F497FF10C0F8CFEB
:1029A0008B3F39F49091AB0297FF09C01092AB02B4
:1029B0002DC08C3F21F49091AB021916BCF39FE01F
:1029C000980F983080F421E030E0A90102C0440F54
:1029D000551F9A95E2F7CA0180959091A702892325
:1029E0008093A70213C08D3F21F48091A5028E7FB2
:1029F0000BC08E3F21F48091A5028D7F05C08F3FD3
:102A000029F48091A5028B7F8093A5028091A80272
:102A1000811106C08091A902811102C01092A40206
:102A20008091AA02811106C08091AB02811102C07F
:102A30001092A30208950E9469232091A8022111F7
:102A400004C02091A902222321F09093A202809336
:102A5000A1022091AA02211104C02091AB022223DD
:102A600021F09093A00280939F0286EA92E00C945A
:102A7000D521EF92FF920F931F93CF93DF9300D056
:102A800000D000D0CDB7DEB786E0E6EAF2E0DE01A6
:102A9000119601900D928A95E1F7E090A802F090CE
:102AA000A9020091AA021091AB021092A802109202
:102AB000A9021092AA021092AB02E11003C0FF20FB
:102AC00009F45DC08091A1029091A2020E9481232D
:102AD000AC019091A402992339F020910A0130E0D1
:102AE0002417350758F04BC020910B018AE0289F2E
:102AF000900111242417350718F041C09F3F19F0A9
:102B00009F5F9093A402EE2061F00E94D1131E14E7
:102B100014F09FEF01C091E0989F902D11249093A5
:102B2000A802FF2061F00E94D1131F1414F09FEF40
:102B300001C091E0989F902D11249093A9023091AB
:102B4000A8023323E1F02091A9022223C1F045EB32
:102B50003403C0011124992319F09093A80203C0F3
:102B600081E08093A80235EB2303C001112499234F
:102B700019F09093A90203C081E08093A90201118A
:102B800003C0112309F45DC080919F029091A002BF
:102B90000E948123AC019091A302992339F02091E6
:102BA000060130E02417350758F04BC0209107018B
:102BB0008AE0289F900111242417350718F041C09E
:102BC0009F3F19F09F5F9093A302002361F00E9442
:102BD0001014101614F09FEF01C091E0989F902DF3
:102BE00011249093AA02112361F00E94101411166F
:102BF00014F09FEF01C091E0989F902D11249093C5
:102C0000AB023091AA023323E1F02091AB022223E0
:102C1000C1F045EB3403C0011124992319F09093BE
:102C2000AA0203C081E08093AA0235EB2303C0010E
:102C30001124992319F09093AB0203C081E0809393
:102C4000AB028091A80281110BC08091A902811171
:102C500007C08091AA02811103C08091AB0281114B
:102C60000E941B15EB82FC820D831E8386E0FE0111
:102C70003196A6EAB2E001900D928A95E1F7269688
:102C80000FB6F894DEBF0FBECDBFDF91CF911F917D
:102C90000F91FF90EF900895E6EAF2E086E0DF0101
:102CA0001D928A95E9F71092A4021092A302109245
:102CB000A5020895EF92FF920F931F93CF93DF9396
:102CC0008B01682F11110AC0442329F0E82FF0E08E
:102CD000E15CFC4F6491762F862F75C0212F30E088
:102CE000E82FF0E0442321F0E15CFC4FE491F0E0B8
:102CF00046E0049FC0011124CFEFD0E0BE010E9446
:102D0000CB2A4BEA4603C001479F900D1124800F48
:102D1000911D800F911D982F990F890FAE01421BB5
:102D2000530B4E9FD0014F9FB00D5E9FB00D1124ED
:102D30009B2F189FA0011124452F55278E01041B9E
:102D4000150B0E9FA0010F9F500D1E9F500D1124BB
:102D50007E01E81AF108E29E8001E39E100DF29ECA
:102D6000100D1124212F3327C21BD30BCE9F9001AE
:102D7000CF9F300DDE9F300D112462307105A9F018
:102D800048F46115710569F061307105C9F48B2F44
:102D9000752F0DC06430710581F058F066307105F3
:102DA00079F47E2F8B2F932F0DC0832F7B2F9E2F97
:102DB00009C08E2F7B2F952F05C08E2F732F02C039
:102DC0007E2F852F692FDF91CF911F910F91FF905B
:102DD000EF90089541E00E945A16089508950E94C8
:102DE000EA160895CF93DF93762FE901682F842F99
:102DF0000E94EF16798368838A83DF91CF910895CB
:102E000080910303282F269530E02115310519F410
:102E10008170826005C02532310524F0817088649C
:102E200080930303089588E090E00C946E2BCF927A
:102E3000DF92EF92FF926B017C010E940017B701B5
:102E4000A60188E090E0FF90EF90DF90CF900C9487
:102E50008C2BE3E0F3E083E0808311828FEF8283A9
:102E60008383148260817181828193810C9417170E
:102E70008091030380FF02C08695089580E0089545
:102E800090910703933018F49F5F90930703882372
:102E900051F06091030370910403809105039091B8
:102EA00006030C941717089581E00C944017909135
:102EB0000703992319F0915090930703882351F049
:102EC00060910303709104038091050390910603C0
:102ED0000C941717089581E00C94571770E00C9428
:102EE0003C1F609110018091030380FF0AC0809114
:102EF0000F0123E0829FC0011124885F9C4F0C9436
:102F00006E178091110190911201891780F7E82FB7
:102F1000F0E09F01220F331FE20FF31FE85FFC4F29
:102F20001182108212828F5FF0CF9091030390FF85
:102F300016C09091110120911201921770F4E92F9F
:102F4000F0E0DF01AA0FBB1FEA0FFB1FE85FFC4F99
:102F50008183608342839F5FF0CF0C947117089543
:102F6000CF93DF9300D01F92CDB7DEB790910303CC
:102F700090FF0AC09E012F5F3F4F0E94F2164B81C7
:102F800069818A810E9495170F900F900F90DF91B1
:102F9000CF910895CF93DF93EC01EC81F0E0E65CF4
:102FA000FD4F4491E3E0F3E0628181810E94B0171C
:102FB0008C818F5F8C83DF91CF910895CF93DF93C6
:102FC000EC01E3E0F3E0438162818C810E94B01761
:102FD0008C818F5F8C83DF91CF9108950F931F9326
:102FE000CF93DF9300D01F92CDB7DEB78C018091D5
:102FF000AC0281110AC09E012F5F3F4F4FEF6FEF70
:103000000E94F2168A818093AC02F801848181309B
:1030100051F028F0823061F44091AC020AC08091F6
:10302000AC0240E007C06091AC0240E080E003C029
:1030300040E080E060E00E949517F801848190E014
:10304000019663E070E00E94DF2A84830F900F9066
:103050000F90DF91CF911F910F910895AF92BF9282
:10306000CF92DF92EF92FF920F931F93CF93DF9354
:1030700000D01F92CDB7DEB7182FF62E042FE22E08
:103080009091030390FF6DC0E92FE695AE2FB0E05D
:10309000AE55BE4F8C918093B6029E7F923061F404
:1030A0009E012F5F3F4F812F0E94F2164B81698155
:1030B0008A810E94951743C0823019F4009106035B
:1030C0003EC0863019F41091040339C08930D9F319
:1030D0008931A9F5E9518E2F8170D82EE695F0E05F
:1030E000E65CFC4FA590B490C12CBB246091130109
:1030F000C61618F52C2D30E0A29EC001A39E900D9F
:10310000B29E900D112470E00E94CB2A812FD11025
:1031100002C0860F01C0861B90911101290F311D3D
:10312000A901440F551F240F351F285F3C4F402F26
:103130006F2D0E94F216C394D9CF0E94711710937D
:103140000403F092050300930603EE2051F0609112
:1031500003037091040380910503909106030E947C
:1031600017170F900F900F90DF91CF911F910F9134
:10317000FF90EF90DF90CF90BF90AF900895E3E085
:10318000F3E09181282F4381628188E0890F0C94BC
:103190002E1881E00C94BF18E3E0F3E09181282F12
:1031A0004381628188EF890F0C942E1881E00C9482
:1031B000CC18E3E0F3E0628128E0620F08F46FEFDF
:1031C000282F438181810C942E1881E00C94D9180A
:1031D000E3E0F3E0628128E0621B08F460E0282F5E
:1031E000438181810C942E1881E00C94E818E3E06F
:1031F000F3E0438128E0420F08F44FEF282F62816B
:1032000081810C942E1881E00C94F718E3E0F3E030
:10321000438128E0421B08F440E0282F628181812D
:103220000C942E1881E00C94061920E00C942E18B2
:10323000FF920F931F93CF93DF93EC01F12C0FEFCD
:1032400010E060911301F616F0F4809111012F2D1A
:1032500030E0280F311DC901880F991F280F391F31
:10326000285F3C4F70E0C8010E94DF2A962F8C81B6
:103270004091060360910503F99E800D11240E9480
:10328000F216F394DECF0E9471179A818C8190FF21
:1032900002C08F5F01C081508C83DF91CF911F915D
:1032A0000F91FF900895BF92CF92DF92EF92FF921D
:1032B0000F931F93CF93DF93FC01828180FF02C0A5
:1032C0000FEF01C001E010E080911301181708F022
:1032D00040C080911101C12ED12CE601C80FD11D33
:1032E000CE01880F991FC80FD91FC85FDC4F198204
:1032F00018821A8234E0E32EF12CB12C8091AE02B8
:103300008B0D853014F0837005C087FF03C090914A
:103310001301890F082E000C990BC816D90691F4D9
:10332000809106038E9DA0018F9D500D112455950F
:103330004795559547959E0160910503809104033B
:103340000E94F216B00EF1E0EF1AF108B9F61F5F15
:10335000BBCF0E9471178091AE02013031F4811110
:1033600002C080911301815007C090E001966091E6
:10337000130170E00E94DF2A8093AE02DF91CF91AB
:103380001F910F91FF90EF90DF90CF90BF90089525
:10339000CF938091110190911201891770F4E82F59
:1033A000F0E09F01220F331FE20FF31FE85FFC4F95
:1033B0001182108212828F5FF0CFC0E06091130102
:1033C000C617C0F5EC2FF0E070E0CF010E94DF2AB5
:1033D00020911101820F2091AD02022E000C330BBF
:1033E00090E0E217F307CCF020910E01022E000CC2
:1033F000330B2E173F078CF09C01220F331F820FD7
:10340000931F9C01285F3C4F409106036091050388
:10341000809104030E94F2160BC0FC01EE0FFF1F07
:103420008E0F9F1FFC01E85FFC4F118210821282F9
:10343000CF5FC4CF0E94711720910D018091AD0222
:10344000820F8093AD0290910E01920F90930E0126
:1034500019165CF4082E000C990B4091130150E0F2
:1034600041505109841795071CF0219520930D01B7
:10347000CF9108958F929F92AF92BF92CF92DF9299
:10348000EF92FF920F931F93CF93DF938C01FC0178
:103490004481C42FD0E09E01DE010E94232B9B01BA
:1034A000AC010E94392B6B017C01E0E2F0E0EC1BE7
:1034B000FD0BA5E5B0E09B01AC010E94392B4B014F
:1034C0005C019F01DF010E941B2B9B01AC010E944C
:1034D000442B9B01AC012C0D3D1D4E1D5F1DC501F4
:1034E000B4010E94F32AC22FD22F2A3228F4F3E02B
:1034F0002F9F900111240DC025E530E02C1B3109D0
:10350000C901880F991F280F391F37FF02C02F5F8D
:103510003F4F35952795C22FC095F12C85E5E82EB4
:10352000ED1A80911301F816C8F4F1FC02C08E2D3B
:1035300001C08D2F909111012F2D30E0290F311DE9
:10354000A901440F551F240F351F285F3C4F4C2FF6
:10355000609105030E94F216F394E3CF0E94711765
:10356000F8018481811102C091E003C0803219F416
:103570009FEF90930C0190910C01890FF8018483C7
:10358000DF91CF911F910F91FF90EF90DF90CF903F
:10359000BF90AF909F908F9008950F931F93CF93FC
:1035A000DF93EC0100E010E080911301282F30E060
:1035B0000217130724F5909111019801290F311D6D
:1035C000A901440F551F240F351F285F3C4F8695D6
:1035D00090E04C81081719071CF4442331F002C015
:1035E000411103C04091060301C040E06091050312
:1035F000809104030E94F2160F5F1F4FD5CF0E94E7
:1036000071178C8190E00196817099278C83DF91EE
:10361000CF911F910F910895E3E0F3E080818E7FB9
:10362000808360817181828193810E94171710923B
:10363000B7022FEF80E792E0215080409040E1F701
:1036400000C000000C94711760910303669570E050
:103650004BE050E084E191E00E944C2B892B19F45F
:1036600081E08093B7020E9469239093B002809317
:10367000AF0208959091030390FF35C091708111BE
:1036800002C0926006C0853210F0986402C0880FB4
:10369000982B90930303662351F06091030370917C
:1036A000040380910503909106030E94171760910F
:1036B0000303669570E04BE050E084E191E00E94E6
:1036C0004C2B892B19F01092B70202C00E94241BC8
:1036D00081E08093B20240910603609105038091DE
:1036E00004030C9415190895682F9091030396957F
:1036F00081E0890F853208F081E00C943A1B81E06B
:103700000C94741B682F9091030396958FEF890F8B
:1037100009F484E20C943A1B81E00C94821B61E072
:103720000C943A1BE3E0F3E080818160808386950E
:103730000C948F1B8091030380FD0C940C1B0C9444
:10374000921B60E00C943A1B8091B50281112EC04F
:103750000E947E0E811104C00E94260F0E9429172C
:103760000E9413176093030370930403809305036F
:10377000909306036E7F61F40E9429170E9413172D
:1037800060930303709304038093050390930603EF
:103790000E9400171092B7028091030380FF03C0BC
:1037A00086950E94A11B81E08093B50208950F9336
:1037B0001F93CF93DF938091B702882309F485C0CC
:1037C0008091B602E0910303E695E81BE093B10215
:1037D000823049F4F0E0EA5CFD4FE491CE2FD0E076
:1037E0000AEC17E149C0863049F4F0E0ED5CFD4F8A
:1037F000E491CE2FD0E00EED17E13EC0893051F4B8
:10380000E695F0E0E05DFD4FE491CE2FD0E008E1D9
:1038100019E132C08F3051F4E695F0E0E35DFD4FE1
:10382000E491CE2FD0E003E519E126C0853149F4BB
:10383000F0E0E65DFD4FE491CE2FD0E008EC19E119
:103840001BC0883181F0833239F4E8E2F2E0C5919F
:10385000D4910EEE17E110C0843251F4C4EFD1E0E0
:103860000DEC1AE109C0C8E2D0E00AE31AE104C095
:10387000C0EDD7E00EEE16E18091B202882361F030
:103880001092B2020E9469239093B0028093AF021B
:103890001092B4021092B3020E946923E091AF0229
:1038A000F091B0028E1B9F0B8F3F9F4770F4EC0F7F
:1038B000FD1FF093B002E093AF028FEA92E0F801AF
:1038C000DF91CF911F910F910994DF91CF911F91BB
:1038D0000F910895882311F0FA0101C0FB010994AA
:1038E000CF93DF93C82FD62F0E9438178C1740F044
:1038F0000E9438178D1720F4DF91CF910C947F1B15
:103900008C2FDF91CF910C948F1B1F93CF93DF935C
:10391000FB0112811111C3C0EC010E94950D82724E
:10392000CD3CFCE5DF0709F49AC0A8F5C73CECE5FF
:10393000DE0709F476C0A8F4C43C9CE5D90709F475
:103940005FC028F4C33CDC4509F457C054C0C53CF3
:103950009CE5D90709F459C0C63CDC4509F45CC0B4
:103960004AC0CA3CFCE5DF0709F46AC050F4C83C11
:10397000ECE5DE0709F45AC0C93CDC4509F45BC03C
:103980003AC0CB3C9CE5D90709F45FC0CC3CDC4590
:1039900009F460C030C0C23DFCE5DF0709F46FC028
:1039A00088F4CF3C9CE5D90709F460C008F45CC0FA
:1039B000C03DFCE5DF0709F45CC0C13DDC4509F40E
:1039C0005BC019C0C53D9CE5D90709F460C050F43F
:1039D000C33DFCE5DF0709F455C0C43DDC4509F4EF
:1039E00054C009C0C63D9CE5D90709F455C0CE3581
:1039F000DD4509F454C011E052C00E949A1B4FC02B
:103A00004CE85BE16FE77BE104C04FE75BE16CE80A
:103A10007BE10E946A1C43C046ED58E169EC78E105
:103A2000F8CF49EC58E166ED78E1F3CF44EF58E187
:103A300065EE78E1EECF45EE58E164EF78E1E9CF4D
:103A400042E159E163E079E1E4CF43E059E162E129
:103A500079E1DFCF4BE657E164E577E1DACF44E582
:103A600057E16BE677E1D5CF81E017C065E082E0F2
:103A700010C068E086E00DC06EE089E00AC064E135
:103A80008FE007C067E185E104C088E106C062E21B
:103A900089E10E94701C03C083E20E948F1B812F6A
:103AA000DF91CF911F91089586E090E00C94662BF2
:103AB000682F86E090E00C947A2B80911403847038
:103AC0008961809314030C94581D0E947E0E81110D
:103AD00004C00E94260F0E945D1D0E94541D809309
:103AE0001403282F26952695269530E0243031059D
:103AF00024F087708861809314038091140380FF01
:103B000004C086958695869501C080E00C94761E4B
:103B100020911403822F869586958695482F50E034
:103B20004330510554F48F5F982F990F990F990FD7
:103B3000822F8770892B80931403809114038160F6
:103B4000809314030E94581D8091140386958695D6
:103B500086950C94761E80911403982F96959695D1
:103B60009695A1F0915E990F990F990F8770892B07
:103B700080931403887F91E009F490E0809114030E
:103B800090FB80F9809314030E94581D80911403C8
:103B90008695869586950C94761E8091140380FDFB
:103BA00013C0816080931403813019F489E08093FD
:103BB0001403809114030E94581D8091140386956C
:103BC000869586950C94761E08958091140380FF47
:103BD00008C08E7F809314030E94581D80E00C94CF
:103BE000761E08958091140380FD0C94E51D0C94BD
:103BF000CD1D90911403892F8695869586958F5FAC
:103C00008F719770843038F4880F880F880F892B54
:103C10008093140302C09093140380911403887F4F
:103C200091E009F490E08091140390FB80F9809377
:103C300014030E94581D80911403869586958695DD
:103C40000C94761E843008F083E0909114039770F2
:103C5000282F220F220F220F922B90931403987F6C
:103C600021E009F420E09091140320FB90F9909357
:103C700014030C94761E0E94221E809114030C944F
:103C8000581D9C01FB018281882349F12E3BFCE5F4
:103C90003F07C9F040F42C3BECE53E0769F02D3BB3
:103CA0003C4561F00895203C9CE5390791F070F0A7
:103CB000213C3C4589F0089583E001C080E00E94EA
:103CC0003B1E80E008950E94AB1DFBCF0E94881D23
:103CD000F8CF0E94F21DF5CF0E94F91DF2CF81E0CE
:103CE0000895279A2F9808952F9808958F929F925C
:103CF000AF92BF92CF92DF92EF92FF920F931F93FA
:103D0000CF93DF93C82F843050F4811109C0809184
:103D10008000877F809380000E94741E06C0C3E0ED
:103D200080918000886080938000A0918600B0918F
:103D300087002C2F30E00E94232B23E030E040E06E
:103D400050E00E94F32A0027122F232F342F012F37
:103D5000122F232F332780918600909187006CE0EB
:103D600070E00E94CB2A6017710730F0C80169E04B
:103D700070E00E94CB2A5EC08091860090918700FF
:103D8000E0908600F0908700E0918600F091870037
:103D9000C6E0D0E0BE010E94CB2A060F171F211DEE
:103DA000311D4801590185E0880C991CAA1CBB1CD7
:103DB0008A95D1F7C701BE010E94CB2A6F01E12C81
:103DC000F12CA7019601260F371F411D511DC5017A
:103DD000B4010E94F32A69017A01E0918600F09112
:103DE0008700CA01B9010E94BB2A9B01AC01DF0117
:103DF0000E94392B9B01AC01C701B6010E94BB2A6E
:103E0000DC01CB012FE0B695A795979587952A956C
:103E1000D1F7009186001091870020E030E008176C
:103E200019072A073B0728F46091860070918700E4
:103E3000CB01BC0170938D0060938C00DF91CF911A
:103E40001F910F91FF90EF90DF90CF90BF90AF90B8
:103E50009F908F90089508950E94711E8AE080932C
:103E6000800089E1809381008FEF9FEF909387001E
:103E7000809386000C94651D879A21B32F7731B308
:103E800030684FB7F894FC01CB01880F991F680F79
:103E9000791F6E0F7F1FE617F70789F0819198E071
:103EA00031BB000000C087FF21BB880F000000C0AD
:103EB00000C000C021BB00C09A9591F7ECCF4FBF66
:103EC0008FE594E00197F1F700C000000895CF93CB
:103ED000DF93EC01FB018281882309F43CC1C430EB
:103EE000FDE5DF0760F4CB3F9CE5D90788F49E0130
:103EF00022503C452431310508F02EC109C0C2369C
:103F0000EDE5DE0729F0C63AFDE5DF0709F024C13B
:103F10000E94910E9093EA028093E902C1318CE5F0
:103F2000D80709F4C6C008F042C0C930ECE5DE0786
:103F300009F49BC000F5C5308CE5D80709F485C0AD
:103F400078F4C330ECE5DE0709F478C008F07AC0F5
:103F5000C230DC4509F0F5C08091E9028160EFC014
:103F6000C7309CE5D90709F478C008F07AC0809181
:103F7000E9028061E4C0CD30FCE5DF0709F487C0C9
:103F800058F4CB309CE5D90709F479C008F07BC020
:103F90008091E90288606FC0CF30FCE5DF0709F44B
:103FA00080C008F082C08091E902877FC8C0CE3F00
:103FB0009CE5D90709F471C000F5C531FCE5DF07C0
:103FC00009F485C068F4C3319CE5D90709F475C0CC
:103FD00008F095C00E9442088091E9028F77AFC037
:103FE000CC3FFCE5DF07A9F108F054C0CB3FDC452E
:103FF00009F0A7C08091EA0240C0C230EDE5DE07BB
:1040000009F489C058F4C1158DE5D80709F45AC0E0
:1040100008F069C08091EA0282602FC0C236EDE5E7
:10402000DE0709F47CC0C63AFDE5DF0709F481C06C
:10403000C330DD4509F085C080E06EC08091E902A3
:1040400082607DC08091E90216C08091E90288609B
:1040500076C08091EA0282604FC08091E90280625E
:104060006EC08091E90280646AC00E94420880911B
:10407000E902806864C0846062C081603DC0809154
:10408000E9028E7F5CC08091E9028D7F58C08091EB
:10409000E90216C08091EA0218C08091EA028D7F81
:1040A0002BC08091E9028F7E4AC08091E9028F7D0A
:1040B00046C08091E9028F7B42C08091E902877FF0
:1040C0008B7F3DC08091EA028D7F8E7F15C08091ED
:1040D000E90282FB222720F991E0922790FB82F9E6
:1040E00090FB83F92CC08091EA02982F90959170F3
:1040F0008E7F892B90FB81F98093EA0222C00E9477
:1041000042088091E90287FB222720F991E092275B
:1041100090FB87F914C081E00E94280F12C08091A3
:10412000E90284FB222720F991E0922790FB84F991
:1041300006C08091E902982F909590FB80F98093BA
:10414000E9028091E9029091EA020E94A20E0E9487
:10415000420880E001C081E0DF91CF910895CF93C4
:10416000DF9386319C4541F5EB010E94950D982F18
:104170008A812091020130910301882379F09A7A93
:1041800081E009F480E08093B802911102C069E2F5
:1041900001C065E3C9010E94A5220AC08091B8024E
:1041A000811102C069E201C065E3C9010E94B02229
:1041B0000E94D70D80E001C081E0DF91CF9108958A
:1041C0000F931F93CF93DF93C42FD22FFC018281D3
:1041D0008823C9F04093BB020E9469239093BA02DE
:1041E0008093B90280E28C0F883008F057C0C77006
:1041F00081E001C0880FCA95EAF7DF91CF911F9146
:104200000F910C949F058091BB02481330C08091A0
:10421000B9029091BA020E948123883C910538F539
:1042200010E21D0FCD17B9F080E28C0F883040F4FA
:10423000C77081E001C0880FCA95EAF70E94A60501
:10424000183028F581E09D2F977001C0880F9A954E
:10425000EAF70E949F05802F0E9496051830F0F41F
:10426000D77081E001C0880FDA95EAF70AC080E2D2
:104270008C0F883098F4C77081E001C0880FCA9510
:10428000EAF7DF91CF911F910F910C94A605802F33
:10429000DF91CF911F910F910C949605DF91CF91F3
:1042A0001F910F9108950F939C01CB01243F4CE582
:1042B000340731F188F4293DFCE53F07D9F02A3D68
:1042C0004CE5340779F1283D3C45A9F506E221EE9D
:1042D00041EE68ED7CE52BC0263FFCE53F07E1F0B1
:1042E000A8F0273F3C4539F507E225EE46EE67EF9B
:1042F0007CE51DC007E225EE45EE69ED7CE517C0C3
:1043000006E221EE40EE64EF7CE511C007E225EE07
:1043100044EE65EF7CE50BC006E221EE42EE66EF6F
:104320007CE505C008E221E045EE6AED7CE50E94EF
:10433000E02080E008C0FC018281882319F01092FF
:10434000BB0201C081E00F9108959093C901809351
:10435000C80108959093C1028093C0020895E0912E
:10436000C002F091C102309721F00190F081E02D60
:10437000099480E00895E091C002F091C102309765
:1043800099F020912B01222359F02091E90227FF77
:1043900007C0DC012C9111962C93119726E02C93E9
:1043A0000280F381E02D09940895E091C002F0911C
:1043B000C102309739F022E0DC012C930480F581B2
:1043C000E02D099408952091BE023091BF02281774
:1043D000390771F09093BF028093BE02E091C00252
:1043E000F091C102309721F00680F781E02D099409
:1043F00008952091BC023091BD022817390771F051
:104400009093BD028093BC02E091C002F091C10282
:10441000309721F00084F185E02D09940895FC0186
:10442000329680912B01882331F08091E90287FF39
:1044300002C09EE101C096E080E0915028F02191F9
:104440002223D9F38F5FF9CF0895662351F120918C
:104450002B012223E9F02091E90227FF19C0462F02
:104460004695469546954E31E0F4677021E030E080
:1044700002C0220F331F6A95E2F7FC01E40FF11D21
:10448000828190E02823392381E0232B69F409C03D
:10449000FC01329608962191621729F0E817F90776
:1044A000D1F780E0089581E008959C01FC013296E7
:1044B0009FEF80E04191461789F09F3F19F4411129
:1044C00001C0982F8F5F8630A9F79F3F39F0F9011F
:1044D000E90FF11D97FDFA956283089508959C01F7
:1044E0002A5F3F4FFC014281461301C012820196B0
:1044F00082179307B9F70895262F269526952695B6
:104500002E3168F4FC01E20FF11D677021E030E00C
:1045100001C0220F6A95EAF78281282B2283089531
:10452000262F2695269526952E3170F4FC01E20F54
:10453000F11D677021E030E001C0220F6A95EAF7B3
:104540002095828128232283089520912B01222304
:1045500029F02091E90227FD0C947C220C9455222D
:1045600020912B01222329F02091E90227FD0C94B0
:1045700090220C946F2220912B01FC013296222371
:1045800031F08091E90287FF02C08EE101C086E030
:10459000DF011D928A95E9F7089508950C94CD22C4
:1045A00083E08093C2020C94CE22811102C081E08C
:1045B00001C082E08093C2020C94CE220C94D522DA
:1045C00081E08093C2020C94CE220C94E0220895E4
:1045D0000C94E7220C94E8220C94E7220C94E72236
:1045E0000C94E722CF930E94EE220E9432130E9485
:1045F000EC22C0E08C2F0E945C12892B29F4CF5F43
:10460000C630C1F780E001C081E0CF9108950895E0
:104610001F920F920FB60F9211248F939F93AF9317
:10462000BF938091C302811113C0809115039091B3
:104630001603A0911703B09118034196A11DB11D57
:104640008093150390931603A0931703B093180358
:10465000BF91AF919F918F910F900FBE0F901F90C0
:10466000189580911D03843031F10E94EF03109260
:10467000C30220E488E190E00FB6F894A8958093F7
:1046800060000FBE2093600083B7817F846083BF8A
:1046900083B7816083BF7894889583B78E7F83BF0B
:1046A0000FB6F894A89580916000886180936000AF
:1046B000109260000FBE08950E9442080C94F60309
:1046C00082E084BD93E095BD9AEF97BD80936E0024
:1046D00008952FB7F8948091150390911603A09137
:1046E0001703B09118032FBF08952FB7F894609166
:1046F00015037091160380911703909118032FBF33
:1047000008959C014FB7F89480911503909116037A
:10471000A0911703B09118034FBF821B930B08950C
:1047200078941F920F920FB60F9211248F939F933C
:10473000AF93BF938091150390911603A091170337
:10474000B09118030196A11DB11D8093150390939C
:104750001603A0931703B0931803BF91AF919F91D5
:104760008F910F900FBE0F901F90189581E080934E
:10477000E00080E28093D8001092C9008FE19EE4AF
:104780000197F1F700C0000087E090EBDC01809317
:10479000260390932703A0932803B09329039CE05A
:1047A00088E10FB6F894A895809360000FBE9093AF
:1047B0006000FFCF8091E7020895089522E02093E2
:1047C000E9002FEF3091E800215035FD06C035EDAE
:1047D0003A95F1F700002111F5CF2091E80025FF6F
:1047E0000BC040E050E066E070E00E941D26809122
:1047F000E8008E778093E8000895CF93DF932091AF
:104800002B01222339F02091E90227FF03C060E247
:1048100022E002C068E021E02093E9002FEF309110
:10482000E800215035FD06C035ED3A95F1F700005E
:104830002111F5CF2091E80025FF1DC0EC018091EA
:104840002B01811105C040E050E068E070E003C03A
:1048500070E040E050E0CE010E941D268091E8000B
:104860008E778093E80080E2FE01A7ECB2E0019031
:104870000D928A95E1F7DF91CF9108958093C4025C
:104880007093C6026093C50280911D03843001F5C8
:1048900082E08093E9008FEF9091E800815095FDD0
:1048A00006C095ED9A95F1F700008111F5CF809142
:1048B000E80085FF0DC040E050E063E070E084EC6C
:1048C00092E00E941D268091E8008E778093E80098
:1048D0000895BC0184E00C943E24BC0183E00C9458
:1048E0003E2480911C03811109C00E94AE270E94C2
:1048F0000B288091E20084608093E200089510927A
:104900001C0308950C94E5226091190381E0611164
:1049100001C080E00C94D02290911D0381E094307E
:1049200009F080E0609119030C94D52242E061EC1B
:1049300081E00E94272742E261EC82E00E94272763
:1049400090911D0381E0943009F080E0609119039B
:104950000C94DE2280911F03833009F461C030F48F
:10496000813071F0823009F49AC008958A3009F4D8
:1049700086C08B3009F46CC0893009F0A8C020C013
:1049800080911E03813A09F0A2C08091E800877FE0
:104990008093E8008091220390912303892B21F4D6
:1049A00060E287EC92E003C060E080E090E070E0BD
:1049B0000E9468268091E8008B778093E800089534
:1049C00080911E03813209F082C080912203909170
:1049D0002303029708F07BC08091E800877F8093D3
:1049E000E8008091E80082FD05C080911D038111DF
:1049F000F8CF6DC02091F3008091F20090E0922BEF
:104A0000029731F48091F100813011F0863021F469
:104A10008091F1008093E7028091E8008B7753C08A
:104A200080911E03813A09F052C080912203909137
:104A30002303892B09F04BC08091E800877F809386
:104A4000E8008091E80080FFFCCF80912B0136C008
:104A500080911E038132D9F5809122039091230326
:104A6000892BA9F58091E800877F8093E8000E9458
:104A70005C278091200380932B010C944208809145
:104A80001E03813221F58091E800877F8093E80042
:104A90000E945C27809121038093E8020895809111
:104AA0001E03813AA1F48091E800877F8093E8009B
:104AB0008091E80080FFFCCF8091E8028093F100B4
:104AC0008091E8008E778093E8000C945C2708952D
:104AD00084B7877F84BF0FB6F894A8958091600053
:104AE000886180936000109260000FBE90E080E8C3
:104AF0000FB6F89480936100909361000FBE0C9400
:104B0000E0220E94AE270E940B28E2EEF0E08081B6
:104B10008460808378940C94A02A8FE191E00C94B7
:104B2000AA2180911D038530A9F480911D03853051
:104B300079F40E94312380911B038823B1F30E94F2
:104B4000F222882391F30E9407260E944208EDCFAB
:104B50000C945C23089508950C94AE25292F3327D7
:104B600023303105C9F060F42130310581F0223065
:104B7000310509F044C08BE390E02DE634E043C0FA
:104B800021323105E1F02232310549F138C082E1AC
:104B900090E028EA34E037C099278130910549F048
:104BA00028F0029761F5EFE3F4E005C0E9E6F4E0F0
:104BB00002C0EDE4F4E0849190E09F0124C061150F
:104BC000710541F061307105D1F489E090E028E988
:104BD00034E019C089E090E02FE734E014C061159B
:104BE000710541F06130710551F486EB90E02AEBDC
:104BF00034E009C080E490E020E735E004C080E0C4
:104C000090E020E030E0FA0131832083089580E1D4
:104C100089BD82E189BD09B400FEFDCF8091D80035
:104C20008F7D8093D8008091E00082608093E000C7
:104C30008091E00081FDFCCF0895CF92DF92EF924A
:104C4000FF920F931F93CF93DF93EC018B017A01B7
:104C50000E947B27811133C0E114F10439F0F70180
:104C600080819181081B190BC80FD91FC12CD12C31
:104C70000115110519F18091E80085FD16C080919C
:104C8000E8008E778093E800E114F10449F0F70121
:104C900080819181C80ED91ED182C08285E00FC06B
:104CA0000E947B27882321F30AC089918093F10019
:104CB00001501109FFEFCF1ADF0ADACF80E0DF9150
:104CC000CF911F910F91FF90EF90DF90CF900895BB
:104CD00020912403309125032617370748F06115EA
:104CE000710539F42091E8002E772093E80001C087
:104CF000B901FC0120E06115710579F180911D0376
:104D00008823F1F18530F1F18091E80083FD3CC00A
:104D10008091E80082FD2EC08091E80080FFEBCFFB
:104D20002091F3008091F20090E0922B61157105C3
:104D300051F08830910538F421912093F1006150B1
:104D400071090196F3CF21E0089709F020E08091E6
:104D5000E8008E778093E800CECF2111CFCF0AC034
:104D600080911D03882361F0853061F08091E80017
:104D700083FD0AC08091E80082FFF2CF80E00895B1
:104D800082E0089583E0089581E00895209124034E
:104D9000309125032617370748F06115710539F45E
:104DA0002091E8002E772093E80001C0B901FC01B2
:104DB00020E06115710591F180911D03882309F4AC
:104DC00040C0853009F43FC08091E80083FD3DC0BC
:104DD0008091E80082FD2FC08091E80080FFE9CF3C
:104DE0002091F3008091F20090E0922B6115710503
:104DF00059F08830910540F424912093F1003196C8
:104E0000615071090196F2CF21E0089709F020E086
:104E10008091E8008E778093E800CBCF2111CCCF32
:104E20000AC080911D03882361F0853061F0809174
:104E3000E80083FD0AC08091E80082FFF2CF80E0A5
:104E4000089582E0089583E0089581E00895982F01
:104E5000973068F59093E900981739F07091EC005D
:104E60002091ED005091F00003C0242F762F50E0E8
:104E700021FD02C09F5FECCF3091EB003E7F30936D
:104E8000EB003091ED003D7F3093ED003091EB0071
:104E900031603093EB007093EC002093ED00509361
:104EA000F0002091EE0027FDE5CF80E008958F709F
:104EB0008093E90081E0089580911E0387FF11C06F
:104EC0008091E80082FD05C080911D038111F8CF1B
:104ED00011C08091E8008B770BC080911D0388235F
:104EE00049F08091E80080FFF8CF8091E8008E774C
:104EF0008093E80008952091E4003091E50095E664
:104F00004091EC00842F817040FF23C08091E80025
:104F100080FD1DC080911D03882399F0853099F094
:104F20008091EB0085FD11C04091E4005091E500B7
:104F30002417350729F3915011F09A01E1CF84E04D
:104F4000089582E0089583E0089581E0089580E067
:104F500008954091E80042FFDDCF08950E941C288B
:104F60000E942428E0EEF0E0808181608083E8EDFB
:104F7000F0E080818F77808319BCA7EDB0E08C9141
:104F80008E7F8C9380818F7E808310921C03089586
:104F90000F931F93CF93DF930E941C280E94242815
:104FA000C8EDD0E088818F77888388818068888386
:104FB00088818F7D888319BC10921D03109219037C
:104FC00010921B0310921A0300EE10E0F80180818A
:104FD0008B7F808388818160888342E060E080E00D
:104FE0000E942727E1EEF0E080818E7F8083E2EE51
:104FF000F0E0808181608083808188608083F80117
:1050000080818E7F8083888180618883DF91CF91CA
:105010001F910F910895E8EDF0E080818F7E8083ED
:10502000E7EDF0E080818160808384E082BF81E0F1
:1050300080931C030C94C827E8EDF0E080818E7FFC
:1050400080831092E20008951092DA001092E1003D
:1050500008951F920F920FB60F9211242F933F9332
:105060004F935F936F937F938F939F93AF93BF9370
:10507000EF93FF938091E10082FF0BC08091E200EB
:1050800082FF07C08091E1008B7F8093E1000E9446
:105090009F2A8091DA0080FF1FC08091D80080FF96
:1050A0001BC08091DA008E7F8093DA008091D90056
:1050B00080FF0DC080E189BD82E189BD09B400FE99
:1050C000FDCF81E080931D030E94712405C019BCAF
:1050D00010921D030E947F248091E10080FF19C07F
:1050E0008091E20080FF15C08091E2008E7F809366
:1050F000E2008091E20080618093E2008091D8001C
:1051000080628093D80019BC85E080931D030E94C3
:1051100084248091E10084FF30C08091E20084FF0C
:105120002CC080E189BD82E189BD09B400FEFDCFBC
:105130008091D8008F7D8093D8008091E1008F7E90
:105140008093E1008091E2008F7E8093E200809165
:10515000E20081608093E20080911903882311F0BE
:1051600084E007C08091E30087FD02C081E001C0B8
:1051700083E080931D030E948C248091E10083FFD3
:1051800029C08091E20083FF25C08091E100877FE4
:105190008093E10082E080931D03109219038091B7
:1051A000E1008E7F8093E1008091E2008E7F80930A
:1051B000E2008091E20080618093E20042E060E0E2
:1051C00080E00E9427278091F00088608093F000A3
:1051D0000E948224FF91EF91BF91AF919F918F9197
:1051E0007F916F915F914F913F912F910F900FBEE3
:1051F0000F901F9018951F920F920FB60F921124C7
:105200002F933F934F935F936F937F938F939F93CE
:10521000AF93BF93CF93DF93EF93FF93C091E900D8
:10522000CF708091EC00D82FD17080FDD0E8109223
:10523000E9008091F000877F8093F00078940E94CD
:105240003F291092E9008091F00088608093F0007F
:10525000CD2BCF70C093E900FF91EF91DF91CF91FB
:10526000BF91AF919F918F917F916F915F914F917E
:105270003F912F910F900FBE0F901F9018951F9385
:10528000CF93DF93CDB7DEB7AA970FB6F894DEBF02
:105290000FBECDBFEEE1F3E08091F100819323E0FA
:1052A000E632F207C9F70E94AA248091E80083FF42
:1052B0002EC180911E0390911F03492F50E04A3068
:1052C000510508F024C1FA01EE59FF4F0C94152B3B
:1052D000803821F0823809F01AC108C080911A0381
:1052E00090911B03992389F082600FC08091220363
:1052F0008F70873008F00BC18093E9008091EB003C
:1053000085FB882780F91092E9009091E800977F4B
:105310009093E8008093F1001092F100D1C0282F03
:105320002D7F09F0F4C0882319F0823061F0EFC0BE
:1053300080912003813009F0EAC0933009F080E0C9
:1053400080931B032EC08091200381112AC080917D
:1053500022038F702FEF280F263008F0D8C08093DB
:10536000E9002091EB0020FF1CC0933021F48091D4
:10537000EB00806214C09091EB0090619093EB0081
:1053800021E030E0A90102C0440F551F8A95E2F7E1
:105390004093EA001092EA008091EB0088608093CD
:1053A000EB001092E9008091E800877F8093E8008D
:1053B0000E945C27ACC08111AAC0109120031F7706
:1053C0008091E3008078812B8093E3008091E80056
:1053D000877F8093E8000E945C278091E80080FF2F
:1053E000FCCF8091E30080688093E300111102C03C
:1053F00082E001C083E080931D0389C08058823021
:1054000008F085C080912003909121038C3D53E0EA
:10541000950779F583E08A838AE289834FB7F89408
:10542000DE01139620E03EE051E2E32FF0E05093DE
:105430005700E49120FF03C0E295EF703F5FEF70EB
:105440008E2F90E0EA3010F0C79601C0C0968D9381
:105450009D932F5F243149F74FBF8091E800877FEC
:105460008093E8006AE270E0CE0101960E9468260F
:1054700016C06091220370912303AE014F5F5F4F0E
:105480000E94AC25BC01892B09F441C09091E80031
:10549000977F9093E80089819A810E94C626809127
:1054A000E8008B778093E80032C0803881F58091E6
:1054B000E800877F8093E800809119038093F100D2
:1054C0008091E8008E7772CF811121C080912003F6
:1054D0009091210399270297D4F48091E800877F67
:1054E0008093E80080912003809319030E945C2739
:1054F00080911903811106C08091E30087FD02C0ED
:1055000081E001C084E080931D030E949624809175
:10551000E80083FF0AC08091E800877F8093E8005D
:105520008091EB0080628093EB00AA960FB6F8940E
:10553000DEBF0FBECDBFDF91CF911F9108950895BB
:10554000CF9380911D038823A1F0C091E900CF7013
:105550009091EC00892F817090FD80E8C82B10920B
:10556000E9008091E80083FD0E943F29CF70C0933D
:10557000E900CF910895DB018F939F930E94392B0F
:10558000BF91AF91A29F800D911DA39F900DB29FDF
:10559000900D11240895AA1BBB1B51E107C0AA1F3F
:1055A000BB1FA617B70710F0A61BB70B881F991FC4
:1055B0005A95A9F780959095BC01CD01089597FB68
:1055C000072E16F4009407D077FD09D00E94CB2A4D
:1055D00007FC05D03EF4909581959F4F08957095F6
:1055E00061957F4F0895A1E21A2EAA1BBB1BFD01F6
:1055F0000DC0AA1FBB1FEE1FFF1FA217B307E407B2
:10560000F50720F0A21BB30BE40BF50B661F771F09
:10561000881F991F1A9469F76095709580959095E9
:105620009B01AC01BD01CF010895EE0FFF1F059056
:10563000F491E02D09940E94232B332312F48A1B4A
:105640009B0B0C94342BA29FB001B39FC001A39F6E
:10565000700D811D1124911DB29F700D811D1124AB
:10566000911D08950E94232BB7FF0895821B930B71
:1056700008950E94232BA59F900DB49F900DA49F89
:10568000800D911D11240895B7FF0C94392B0E94B1
:10569000392B821B930B0895FC014150504030F090
:1056A00001900616D1F73197CF01089588279927E1
:1056B0000895FB01DC0104C08D910190801921F453
:1056C00041505040C8F7881B990B0895F999FECFB7
:1056D00092BD81BDF89A992780B50895A6E1B0E002
:1056E00044E050E00C94A02BA8E1B0E042E050E090
:1056F0000C94A02B262FF999FECF92BD81BDF89A6C
:10570000019700B4021639F01FBA20BD0FB6F89405
:10571000FA9AF99A0FBE08950396272F0E947B2BC1
:105720000E947A2B252F0E947B2B242F0C947B2BFD
:105730000196272F0E947B2B0C947A2BDC01CB0146
:10574000FC01F999FECF06C0F2BDE1BDF89A319691
:1057500000B40D9241505040B8F70895F894FFCF2F
:10576000C8006502280850011E0A14010101020048
:105770000400040401191A1B1C1D1E1F202122DA1B
:1057800023FD23DE236D246924DD2301E200E900EB
:10579000EA00B500B600B700CD008301CC008A0155
:1057A00092019401210223022402250226022702EB
:1057B0002A02B300B4006F007000818283E200E926
:1057C00000EA00B500B600B700CD008301CC008A26
:1057D00001920194012102230224022502260227BC
:1057E000022A02B300B4006F007000818283F5F4D6
:1057F000F1F0309593969734353666929091313228
:10580000C633000102020202060606090909090957
:10581000090F0F0F0F0F0F15151518191919191951
:085820001919191919232400BC
:00000001FF
